:1000000000308A00932B0000FF00030E8301A10043
:100010000A08A0008A010408A2007708A300780853
:10002000A4007908A5007A08A6007B08A70083131E
:1000300083128B1E1D280B1936288C308400801EDD
:1000400023288C1A3928220884002308F700240862
:10005000F8002508F9002608FA002708FB00200808
:100060008A00210E8300FF0E7F0E09008A110A12FA
:10007000C6288A110A12A0280A108A100A118207BB
:100080005234533434343834353400340A108A103E
:100090000A11820753347434613472347434003476
:1000A0000A108A100A11820743346F346D346D349C
:1000B00061346E34643400340A108A100A118207E5
:1000C0004534723472346F34723400348C1E6628B6
:1000D0001808AE001A08F800AE1C7028181218167E
:1000E0000000003483160612831206160C1E7628B2
:1000F00083163C08831299000000831606128312AF
:1001000006168316981886288312812806128312F1
:100110000612003483168612831286168316061280
:100120008312061600348C1E9728662093288316A7
:100130008612831286128316061283120612003468
:1001400031308316B800B901BA01BB0183126620B1
:1001500078088316AD002D080D3C031DBA280D301C
:10016000BC00831272200A308316BC0083127220F6
:10017000C228831683128A2083162D08BC0083129E
:10018000722093208C128A110A122328D20A031992
:10019000D30ACC0BF4280130C8070318C90A031985
:1001A000CA0A0319CB0A48080139F700F801F90116
:1001B000FA01F708031DE528F808031DE528F908EA
:1001C000031DE528FA080319EC288711C11141081D
:1001D00083168700F12883128715C1114108831601
:1001E00087000F308312CC000B118A110A122328CA
:1001F00075308400000803190C290130F800F7015C
:10020000F70B0029F80BFF284A30F700F70B0629F7
:1002100000000000800BFD280034EC016B086C0727
:100220008400800803191629EC0A0E29ED018A20A2
:10023000EF01EE016F08013C031C3A29031D24293C
:100240006E08903C031C3A29C117410883168700A9
:100250008312871F2E29EF01EE0133291030F7009A
:10026000F70B30290000ED08031D6400EE0A0319A6
:10027000EF0A1A29A8018B1BA8178B139320A81B20
:100280008B170130ED004708EE006C08EF006B089B
:10029000F00074108A20F1017108043C031CA629A7
:1002A0002E1330306D07F500A8018B1BA8178B1398
:1002B00075088316BC0083127220A81B8B17303080
:1002C0006E07F500A8018B1BA8178B137508831602
:1002D000BC0083127220A81B8B1730306F07F5000B
:1002E000A8018B1BA8178B1375088316BC008312FB
:1002F0007220A81B8B17F2016E086D066F06F300C3
:100300006F08720203189A29700884000008F30627
:10031000700884000008F500A8018B1BA8178B1338
:1003200075088316BC0083127220A81B8B17F00A75
:10033000F20A80292E1BA1296E08F500F8207414FA
:10034000A6296E08F500F820F10A4C29A8018B1B9C
:10035000A8178B139320A81B8B170030741801303B
:10036000F800F808031DB8290A30F500F8204129E3
:1003700000347208F80171020318C1297108F700EE
:10038000CD29F7010830F300F10DF70D720877025F
:100390000318F700F80DF30BC429003420306C1E4D
:1003A0003030ED006B08F700EB1FDD29F709F70A85
:1003B0007708EB002D30ED00EC176B08F10064308E
:1003C000F200B9217708EB0030307807EE006B08B7
:1003D000F1000A30F200B92130307707F0003030F8
:1003E0007807EF006D08F700EC1DF829EC1F6C1181
:1003F0006C1A052AEC1F202A6C19202A7708EE00B7
:10040000EC18202A7708EF00202A30306E02031DF6
:10041000202A7708EE002030ED00EC1D132A6C1125
:10042000EC14EC1FEC1030306F02031D202A77080B
:10043000EF002030EE00EC1D132AEC10EC1F6C10C6
:100440006C1D2D2AA8018B1BA8178B136D08831612
:10045000BC0083127220A81B8B17EC1C3A2AA8013F
:100460008B1BA8178B136E088316BC008312722097
:10047000A81B8B176C1C472AA8018B1BA8178B1372
:100480006F088316BC0083127220A81B8B17A8016B
:100490008B1BA8178B1370088316BC008312722065
:1004A000A81B8B170034A8018B1BA8178B13932054
:1004B000A81B8B17AF01B001B101B301B2018316C4
:1004C0008C16C03083128B048A110A123E2CEE085F
:1004D00003196D2AB2080319672AB208031D742A8A
:1004E0000030F8008A2A8A2A30306D073502031D51
:1004F000862A6B088400380880006C08840037085E
:100500008000B2010130F8008A2A8A2AB201003044
:10051000F8008A2A8A110A125D2C8B12CB01CA01BB
:10052000C901C8010F30CC008B168A110A128A2C1F
:100530008B124B08D0004A08CF004908CE0048086B
:10054000CD004C080F3CD1008B168A110A129B2C4F
:10055000F701F801F901FA018316A801A901AA011E
:10056000AB0127082604250424040319E72A2030B8
:10057000AC000310A00DA10DA20DA30DA80DA90D97
:10058000AA0DAB0D27082B02031DD02A26082A022C
:10059000031DD02A25082902031DD02A2408280279
:1005A000031CE12A2408A8022508031C250FA90220
:1005B0002608031C260FAA022708031C270FAB02DC
:1005C0000314F70DF80DF90DFA0DAC0BB92A000064
:1005D000A8308400831200340408EF00EE1FFD2AC7
:1005E000EF03EF16EB09EC09ED09EE09EB0A03192D
:1005F000EC0A0319ED0A0319EE0A3B30F4009A30B5
:10060000F300CA30F200F1010A30F0006E088316E0
:10061000A30083126D088316A20083126C08831650
:10062000A10083126B088316A0007408A70073084A
:10063000A6007208A5007108A4008312A822000871
:10064000EB00840A0008EC00840A0008ED00840A2C
:100650000008EE00F708031D402B7008013A03194B
:10066000402B6F080319422B0F39700203193A2BE4
:100670000318762BEF1B762B6F1B422B20306A2B37
:100680002030EF05EF1E552BEF127708EF00A80181
:100690008B1BA8178B132D308316BC00831272207E
:1006A000A81B8B176F08F700EF013030EF1E6A2B85
:1006B000EF127708EF00A8018B1BA8178B132D30C2
:1006C0008316BC0083127220A81B8B176F08F700DB
:1006D000EF013030F707A8018B1BA8178B137708A1
:1006E0008316BC0083127220A81B8B177408831614
:1006F000A3007308A2007208A1007108A000A7015E
:10070000A601A5010A30A4008312A8227A08F400E9
:100710007908F3007808F2007708F100F00B062B57
:100720008A110A12BA2C84011F308305831606121F
:1007300083120612193083169900263098009030E3
:100740008312980083161F149F141F159F110730E2
:100750009C008312A9010130AA00AB01AC01AD01DC
:10076000AE01BA01BB01BC01BD01BE01BF01C001A8
:10077000FF30C100C201C301C401C701D201D301CE
:10078000D80159108711C1114108831687008312BF
:10079000C114410883168700003083128718013086
:1007A000F7000310770DEC00411441088316870011
:1007B00000308312071801306C04C700A8018B1B9E
:1007C000A8178B130A308316BC0083127220A81B53
:1007D0008B178715C1114108831687008312EB011F
:1007E000EC015B3084006B0884076C083C208000BF
:1007F00000380319FE2BEC0AEB0AF12B0F30CC006A
:1008000081010730F700F71D0D2C07308101813081
:1008100084000008C0390F388000640081308400F3
:100820000008C039770480005B30EB000D21A8017F
:100830008B1BA8178B1349308316BC0083127220C0
:10084000A81B8B17A8018B1BA8178B13443083168A
:10085000BC0083127220A81B8B17A8018B1BA81742
:100860008B133D308316BC0083127220A81B8B179C
:100870004708EB001F30EC00CE21532AA8018B1B48
:10088000A8178B130D308316BC0083127220A81B8F
:100890008B17A8018B1BA8178B130A308316BC007B
:1008A00083127220A81B8B178B164630EB00453045
:1008B000EC004708ED00EE01672AF8080319D32C75
:1008C000EB01EC015B3084006B0884076C08462068
:1008D0008000003803196F2CEC0AEB0A622C5B30A5
:1008E000EB000D214508533A03197A2C103A0319ED
:1008F000942CC02CEB01EC015B3084006B08840766
:100900006C084620800000380319892CEC0AEB0A99
:100910007C2C8D2A071641124108831687005B3014
:100920008312EB000D21D32C0712411241088316CC
:1009300087008312982AEB016B085020EB0AF7001E
:10094000A8018B1BA8178B1377088316BC00831292
:100950007220A81B8B1707306B02031D9C2C4130A3
:1009600084005008EE004F08ED004E08EC004D08E2
:10097000EB00EC2A5108EB001F30EC00CE21D32C09
:10098000EB01EC015B3084006B0884076C085C2091
:10099000800000380319CF2CEC0AEB0AC22C5B3024
:0A09A000EB000D21D32C552C630051
:02400E00713F00
:00000001FF
